:100000000C944A000C9465000C9465000C946500F7
:100010000C9465000C9465000C9465000C946500CC
:100020000C9465000C9465000C9465000C946500BC
:100030000C9465000C9465000C9465000C946500AC
:100040000C9465000C9465000C9465000C9465009C
:100050000C9465004E0296029E02B7020D03E40264
:10006000480361038503B803E0031C043E045F04F6
:100070007804A004DD04F6042705620574058D05E7
:10008000B705D705FF0516062D0646066606820645
:100090009506AB0611241FBECFE5D4E0DEBFCDBF71
:1000A00011E0A0E6B0E0E6E8FFE002C005900D92A6
:1000B000A83FB107D9F711E0A8EFB1E001C01D9248
:1000C000AD3FB107E1F70C94F9060C9400000097DE
:1000D00079F006C0000000000000000000000000F1
:1000E000000000000000000000000000019791F7F0
:1000F00008950895009731F0E0EAFFE03197F1F7B5
:100100000197D1F708955F9BFECF8CB19927089591
:100110005D9BFECF8CB90895803118F081E090E0AE
:10012000089528B32F70992734E0880F991F3A95C6
:10013000E1F7282B28BB80E090E008950895982FE0
:100140008FEF84BB95BB089514BA85B399270895A2
:10015000CF93C0E00E948C00892B49F4C09881E0C5
:1001600090E00E9467000E94A400C82FC09A8C2FC4
:100170009927CF9108951F93CF93DF93162F0E9455
:100180008C00EC01892B59F4812F0E949F00C198AB
:1001900081E090E00E946700C19ACE0102C081E038
:1001A00090E0DF91CF911F91089599E693BFBB9A9C
:1001B0001CBE82EA8FBD8DE18EBD81B3806381BBA1
:1001C0001BBC1ABC19BC18BC95BD8F9A13BC0895F2
:1001D000CF93C82F843018F081E090E043C088238B
:1001E00041F4962F882764E670E00E9445076CBFB3
:1001F00037C0833041F4962F882764E670E00E9470
:10020000450763BD2DC086B5E82FFF2787B5992721
:10021000982F8827E82BF92BCF01AA27BB279B0112
:1002200044275527BC01CD010E942607DC01CB01E4
:10023000BC01CD0124E630E040E050E00E946C07B4
:10024000DA01C901F901C13029F4892F99278BBD41
:10025000EABD06C0C23021F4892F992789BDE8BDC7
:1002600080E090E0CF9108959C01832F992787BD6E
:1002700026BD0895EF92FF920F931F938B017A0191
:100280000E943401B80181E00E94E800B70182E0D9
:100290000E94E8001F910F91FF90EF900895982F12
:1002A00087E986B99770906497B9369A3699FECFE8
:1002B00084B1282F332785B19927982F8827282B99
:1002C000392B349A3798C9010895599810BC83E3A3
:1002D00089B986E880BD88E18AB9089588B38360CA
:1002E00088BB87B3836087BB87B3806F87BB14BA33
:1002F00008951ABA0E946E010E9465010E94D500FD
:100300000895CF93DF93EC018881882331F08991A0
:100310000E94880088818823D1F780E090E0DF91F7
:10032000CF910895AF92BF92CF92DF92EF92FF925A
:100330000F931F93992764E670E00E9459077B0191
:100340008C016AE070E0C8010E9459075B016C01F2
:10035000E114F10429F08E2D805D0E94880002C016
:10036000672B21F08A2D805D0E9488008C2D805D96
:100370000E9488001F910F91FF90EF90DF90CF9027
:10038000BF90AF900895BF92CF92DF92EF92FF920D
:100390000F931F93CF93DF93BB24009711F480E357
:1003A0001FC08C01C8EDD1E066E0C62ED12CCC0E6A
:1003B000DD1E68817981C8010E9459077B018C018B
:1003C000672B11F4BB2031F08E2D805D0E948800D8
:1003D00051E0B52E2296CC16DD065CF7802F805DAD
:1003E0000E948800DF91CF911F910F91FF90EF90B5
:1003F000DF90CF90BF90089582ED91E00E9481013F
:100400008BEA91E00E9481011092F9011092F801AB
:1004100008958BEA91E00E94810184EA91E00E94B4
:1004200081018BEA91E00E9481011092F901109202
:10043000F80108958BEA91E00E94810187EA91E03A
:100440000E9481018BEA91E00E9481011092F901E2
:100450001092F80108950F931F93CF93C82F082F80
:100460001127C8010E94AB07892B21F0C8010E9407
:10047000BA07C82F8091F8019091F901AA2797FD3A
:10048000A095BA2FFC01809708F0AFC4E65DFF4F3E
:10049000EE0FFF1F0590F491E02D0994C23739F457
:1004A00082E090E09093F9018093F8019EC4C737F1
:1004B00039F486E090E09093F9018093F80195C4B7
:1004C000C03739F48BE090E09093F9018093F80104
:1004D0008CC4C13639F484E190E09093F9018093A3
:1004E000F80183C4C53639F488E190E09093F901AE
:1004F0008093F8017AC4C83639F48FE190E0909384
:10050000F9018093F80171C4CA3019F0CD3009F0B7
:100510006CC48BEA91E00E94810187EA91E00E941D
:1005200081018BEA91E00E9481015FC4CA3019F019
:10053000CD3009F05AC40E941A0257C4C03211F0DB
:10054000C93039F483E090E09093F9018093F80189
:100550004CC4CA3011F0CD3019F40E941A0245C4BF
:1005600081E090E09093F9018093F8013EC48C2FD4
:1005700099270E94B307892B51F0C053C093FA0109
:1005800084E090E09093F9018093F8012EC4CA3280
:1005900039F485E090E09093F9018093F80125C447
:1005A000C03209F422C4C93009F41FC4CA3011F0A2
:1005B000CD3019F40E941A0218C481E090E09093A3
:1005C000F9018093F80111C4CA3011F0CD30F1F473
:1005D0008BEA91E00E9481011092FA018091FA0168
:1005E0000E94A80099279093FC018093FB010E9430
:1005F000C30180E20E9488008091FA018F5F80939E
:10060000FA01803158F30E940902EFC381E090E0C3
:100610009093F9018093F801E8C3CA3011F0CD300E
:10062000B1F48091FA010E94A80099279093FC01EF
:100630008093FB018BEA91E00E9481018091FB0194
:100640009091FC010E94C3010E940902CEC38C2F2D
:1006500099270E94B307892BA1F09091FA018AE0B3
:10066000989F802D11248C0F80538093FA01803144
:1006700008F4BBC381E090E09093F9018093F80106
:10068000B4C381E090E09093F9018093F801ADC389
:10069000C03211F0C93039F487E090E09093F9014D
:1006A0008093F801A2C3CA3011F0CD3019F40E9432
:1006B0001A029BC381E090E09093F9018093F801C6
:1006C00094C38C2F99270E94B307892B51F0C053F4
:1006D000C093FA0188E090E09093F9018093F801CB
:1006E00084C3C03209F481C3C93009F47EC3CA305F
:1006F00011F0CD3019F40E941A0277C381E090E026
:100700009093F9018093F80170C3C03211F0C930A1
:1007100039F489E090E09093F9018093F80165C382
:100720008C2F99270E94B307892BA1F09091FA0191
:100730008AE0989F802D11248C0F80538093FA01BA
:10074000803108F452C381E090E09093F9018093E6
:10075000F8014BC3CA3011F0CD3019F40E941A02CF
:1007600044C381E090E09093F9018093F8013DC388
:100770000C2F1127C8010E94B307892B69F0005381
:1007800010401093FC010093FB018AE090E09093ED
:10079000F9018093F80129C3C03209F426C3C93096
:1007A00009F423C3CA3011F0CD3019F40E941A02A3
:1007B0001CC381E090E09093F9018093F80115C388
:1007C0000C2F1127C8010E94B307892B09F1209132
:1007D000FB013091FC01C901F3E0880F991FFA95E4
:1007E000E1F7820F931F820F931F800F911FC09715
:1007F0009093FC018093FB018F3F910509F00CF46D
:10080000F4C281E090E09093F9018093F801EDC289
:10081000CA3011F0CD3049F46091FB018091FA01AA
:100820000E94BB000E940902E0C281E090E0909328
:10083000F9018093F801D9C2C03211F0C93039F4FE
:100840008CE090E09093F9018093F801CEC2C63617
:1008500039F480E190E09093F9018093F801C5C2EA
:10086000CA3011F0CD3019F40E941A02BEC281E0E4
:1008700090E09093F9018093F801B7C28C2F8053D8
:10088000843048F48093FA018DE090E09093F90170
:100890008093F801AAC2C03209F4A7C2C93009F492
:1008A000A4C2CA3011F0CD3019F40E941A029DC2C0
:1008B00081E090E09093F9018093F80196C2C032F4
:1008C00011F0C93039F48EE090E09093F9018093F3
:1008D000F8018BC2CA3011F0CD3019F40E941A020F
:1008E00084C281E090E09093F9018093F8017DC289
:1008F0000C2F1127C8010E94B307892B69F0005300
:1009000010401093FC010093FB018FE090E0909366
:10091000F9018093F80169C2C03209F466C2C93096
:1009200009F463C2CA3011F0CD3019F40E941A02E2
:100930005CC281E090E09093F9018093F80155C288
:100940000C2F1127C8010E94B307892B01F12091B8
:10095000FB013091FC01C901E3E0880F991FEA9582
:10096000E1F7820F931F820F931F800F911FC09793
:100970009093FC018093FB01853691050CF435C200
:1009800081E090E09093F9018093F8012EC2CA3083
:1009900011F0CD3059F46091FB017091FC01809110
:1009A000FA010E94E8000E9409021FC281E090E063
:1009B0009093F9018093F80118C2C03211F0C93048
:1009C00039F481E190E09093F9018093F8010DC230
:1009D000CA3011F0CD3019F40E941A0206C281E02B
:1009E00090E09093F9018093F801FFC10C2F11273B
:1009F000C8010E94B307892B69F00053104010937F
:100A0000FC010093FB0182E190E09093F901809357
:100A1000F801EBC1C13239F483E190E09093F90120
:100A20008093F801E2C1C03209F4DFC1C93009F492
:100A3000DCC1CA3011F0CD3019F40E941A02D5C1C0
:100A400081E090E09093F9018093F801CEC10C2FE2
:100A50001127C8010E94B307892B01F12091FB01E6
:100A60003091FC01C90173E0880F991F7A95E1F775
:100A7000820F931F820F931F800F911FC097909337
:100A8000FC018093FB01855C99400CF4AEC181E0D0
:100A900090E09093F9018093F801A7C1CA3011F05A
:100AA000CD3049F48091FB019091FC010E9434010A
:100AB0000E9409029AC181E090E09093F90180932D
:100AC000F80193C1CA3011F0CD3039F484E190E0DF
:100AD0000E9434010E94090288C181E090E0909355
:100AE000F9018093F80181C1C03211F0C93039F4A5
:100AF00085E190E09093F9018093F80176C1CA30C6
:100B000011F0CD3019F40E941A026FC181E090E01B
:100B10009093F9018093F80168C18C2F805388303D
:100B200048F48093FA0186E190E09093F901809374
:100B3000F8015BC1CA3239F487E190E09093F90182
:100B40008093F80152C1C03209F44FC1C93009F491
:100B50004CC1CA3011F0CD3019F40E941A0245C1BF
:100B600081E090E09093F9018093F8013EC1CA3092
:100B700011F0CD30A9F48091FA010E944F019093B9
:100B8000FC018093FB018BEA91E00E94810180913E
:100B9000FB019091FC010E94C3010E94090225C142
:100BA00081E090E09093F9018093F8011EC1CA3072
:100BB00011F0CD30E9F48BEA91E00E9481011092AE
:100BC000FA018091FA010E944F019093FC018093F9
:100BD000FB010E94C30180E20E9488008091FA011B
:100BE0008F5F8093FA01883060F30E940902FDC094
:100BF00081E090E09093F9018093F801F6C0CF3640
:100C000039F489E190E09093F9018093F801EDC007
:100C1000CA3011F0CD3019F40E941A02E6C081E00A
:100C200090E09093F9018093F801DFC0CC3639F45D
:100C30008AE190E09093F9018093F801D6C0CA3020
:100C400011F0CD3019F40E941A02CFC081E090E07B
:100C50009093F9018093F801C8C0C03211F0C930F7
:100C600039F48BE190E09093F9018093F801BDC0D5
:100C7000CA3011F0CD3019F40E941A02B6C081E0DA
:100C800090E09093F9018093F801AFC0C23739F436
:100C90008CE190E09093F9018093F801A6C0CE36E4
:100CA00039F48DE190E09093F9018093F8019DC0B3
:100CB000CA3011F0CD3019F40E941A0296C081E0BA
:100CC00090E09093F9018093F8018FC0CE3639F40B
:100CD0008EE190E09093F9018093F80186C0CA30CC
:100CE00011F0CD3041F48DE08093AB011092AC0156
:100CF0000E9409027AC081E090E09093F90180930C
:100D0000F80173C0CA3011F0CD3041F48AE080930D
:100D1000AB011092AC010E94090267C081E090E033
:100D20009093F9018093F80160C0CA3011F0CD3082
:100D300059F48DE08093AB018AE08093AC0110926E
:100D4000AD010E94090251C081E090E09093F90149
:100D50008093F8014AC0CA3019F0CD3009F03FC085
:100D60008BEA91E00E94810184E890E00E94810179
:100D70008BEA91E00E9481018DEA90E00E9481015E
:100D80008BEA91E00E94810188ED90E00E94810150
:100D90008BEA91E00E94810188E091E00E9481014C
:100DA0008BEA91E00E94810187E391E00E9481013A
:100DB0008BEA91E00E9481018BE591E00E94810124
:100DC0008BEA91E00E9481018AE891E00E94810112
:100DD0008BEA91E00E9481010E94090206C081E035
:100DE00090E09093F9018093F801CF911F910F91BA
:100DF0000895CFE5D4E0DEBFCDBF0E9479018CEC31
:100E000091E00E9481018BEA91E00E94810180EED5
:100E100091E00E9481018BEA91E00E9481018EEABB
:100E200091E00E9481018BEA91E00E94810180E6BD
:100E300090E00E9481018BEA91E00E9481010E9472
:100E4000FC010E9483000E942B02FBCF629FD00115
:100E5000739FF001829FE00DF11D649FE00DF11D75
:100E6000929FF00D839FF00D749FF00D659FF00D24
:100E70009927729FB00DE11DF91F639FB00DE11D11
:100E8000F91FBD01CF0111240895AA1BBB1B51E11D
:100E900007C0AA1FBB1FA617B70710F0A61BB70BEA
:100EA000881F991F5A95A9F780959095BC01CD018F
:100EB000089597FB092E07260AD077FD04D0E5DFB9
:100EC00006D000201AF4709561957F4F0895F6F7CB
:100ED000909581959F4F089597FB092E05260ED07A
:100EE00057FD04D014D00AD0001C38F4509540951A
:100EF000309521953F4F4F4F5F4F0895F6F79095EE
:100F00008095709561957F4F8F4F9F4F0895A1E217
:100F10001A2EAA1BBB1BFD010DC0AA1FBB1FEE1F73
:100F2000FF1FA217B307E407F50720F0A21BB30BBE
:100F3000E40BF50B661F771F881F991F1A9469F73A
:100F400060957095809590959B01AC01BD01CF0196
:100F5000089585FD15C08062992391F4813684F04F
:100F60008B3774F40895992359F480334CF08A3305
:100F70003CF408958F93EFDF8F9109F0806208951C
:060F80009927882708955F
:100F8600245265766973696F6E3A20312E352024B6
:100F9600206169645F6C69622E61746D6567613199
:100FA600362E630052656164202028414944206240
:100FB60075732920202D2D3E205B72525D205B3CEF
:100FC600616464726573733E5D5B2A5D0057726986
:100FD60074652028414944206275732920202D2DEF
:100FE6003E205B77575D203C616464726573733E97
:100FF600203C646174613E0050574D20286475742E
:1010060079206379636C6529202D2D3E205B705015
:101016005D203C616464726573733E203C64757444
:10102600796379636C653E0050574D20286672657A
:101036007175656E63792920202D2D3E205B7050D9
:101046005D5B66465D205B3C6672657175656E63C9
:10105600793E5D5B215D00412F4420202020202029
:1010660020202020202020202D2D3E205B61415D68
:10107600203C616464726573733E00454F4C28657D
:101086006E64206F66206C696E6529202D2D3E20CA
:101096005B65455D5B6F4F5D5B6C4C5D205B3C72D9
:1010A600523E5D5B3C6E4E3E5D0048656C70202096
:1010B60020202020202020202020202D2D3E205BB7
:1010C60068485D004F4B00455252000D0A002452FD
:1010D60065766973696F6E3A20312E346D707720AC
:1010E60024206169645F636D642E630048656C6CDF
:1010F6006F005265616479001027E80364000A00F6
:10110600245265766973696F6E3A20312E34202435
:08111600206D61696E2E63007B
:00000001FF
